 jpeg

 Timestamp is 5356bb41 (Tue Apr 22 11:56:01 2014)

 Preferred load address is 10000000

 Start         Length     Name                   Class
 0001:00000000 0001888cH .text                   CODE
 0002:00000000 0000005cH .idata$5                DATA
 0002:00000060 00002428H .rdata                  DATA
 0002:00002488 00000058H .rdata$debug            DATA
 0002:000024e0 00000004H .rdata$sxdata           DATA
 0002:000024e4 00000004H .rtc$IAA                DATA
 0002:000024e8 00000004H .rtc$IZZ                DATA
 0002:000024ec 00000004H .rtc$TAA                DATA
 0002:000024f0 00000004H .rtc$TZZ                DATA
 0002:000024f4 0000003cH .idata$2                DATA
 0002:00002530 00000014H .idata$3                DATA
 0002:00002544 0000005cH .idata$4                DATA
 0002:000025a0 0000014cH .idata$6                DATA
 0002:000026f0 00000631H .edata                  DATA
 0003:00000000 00000004H .CRT$XCA                DATA
 0003:00000004 00000004H .CRT$XCZ                DATA
 0003:00000008 00000004H .CRT$XIA                DATA
 0003:0000000c 00000004H .CRT$XIZ                DATA
 0003:00000010 00000004H .data                   DATA
 0003:00000014 00000070H .bss                    DATA
 0004:00000000 00000058H .rsrc$01                DATA
 0004:00000060 00000310H .rsrc$02                DATA

  Address         Publics by Value              Rva+Base     Lib:Object

 0000:00000000       __except_list              00000000     <absolute>
 0000:00000001       ___safe_se_handler_count   00000001     <absolute>
 0000:00009876       __ldused                   00009876     <absolute>
 0000:00009876       __fltused                  00009876     <absolute>
 0001:00000570       _sun_jpeg_init_source      10001570 f   jpegdecoder.obj
 0001:00000570       _imageio_init_source       10001570 f   imageioJPEG.obj
 0001:00000590       _imageio_fill_input_buffer 10001590 f   imageioJPEG.obj
 0001:000006b0       _imageio_skip_input_data   100016b0 f   imageioJPEG.obj
 0001:00000810       _imageio_term_source       10001810 f   imageioJPEG.obj
 0001:000008a0       _read_icc_profile          100018a0 f   imageioJPEG.obj
 0001:00000ba0       _Java_com_sun_imageio_plugins_jpeg_JPEGImageReader_initReaderIDs@20 10001ba0 f   imageioJPEG.obj
 0001:00000cf0       _Java_com_sun_imageio_plugins_jpeg_JPEGImageReader_readImageHeader@24 10001cf0 f   imageioJPEG.obj
 0001:00000f60       _Java_com_sun_imageio_plugins_jpeg_JPEGImageReader_setOutColorSpace@20 10001f60 f   imageioJPEG.obj
 0001:00000f90       _Java_com_sun_imageio_plugins_jpeg_JPEGImageReader_readImage@80 10001f90 f   imageioJPEG.obj
 0001:00001700       _Java_com_sun_imageio_plugins_jpeg_JPEGImageReader_abortRead@16 10002700 f   imageioJPEG.obj
 0001:00001730       _Java_com_sun_imageio_plugins_jpeg_JPEGImageReader_resetLibraryState@16 10002730 f   imageioJPEG.obj
 0001:00001960       _Java_com_sun_imageio_plugins_jpeg_JPEGImageWriter_initWriterIDs@16 10002960 f   imageioJPEG.obj
 0001:00001a40       _Java_com_sun_imageio_plugins_jpeg_JPEGImageWriter_writeTables@28 10002a40 f   imageioJPEG.obj
 0001:00001b80       _Java_com_sun_imageio_plugins_jpeg_JPEGImageWriter_writeImage@116 10002b80 f   imageioJPEG.obj
 0001:00002390       _Java_com_sun_imageio_plugins_jpeg_JPEGImageWriter_abortWrite@16 10003390 f   imageioJPEG.obj
 0001:000025b0       _Java_com_sun_imageio_plugins_jpeg_JPEGImageReader_setSource@16 100035b0 f   imageioJPEG.obj
 0001:00002600       _Java_com_sun_imageio_plugins_jpeg_JPEGImageReader_resetReader@16 10003600 f   imageioJPEG.obj
 0001:00002690       _Java_com_sun_imageio_plugins_jpeg_JPEGImageWriter_setDest@16 10003690 f   imageioJPEG.obj
 0001:000026e0       _Java_com_sun_imageio_plugins_jpeg_JPEGImageWriter_resetWriter@16 100036e0 f   imageioJPEG.obj
 0001:000028d0       _Java_com_sun_imageio_plugins_jpeg_JPEGImageReader_initJPEGImageReader@8 100038d0 f   imageioJPEG.obj
 0001:00002a60       _Java_com_sun_imageio_plugins_jpeg_JPEGImageReader_disposeReader@16 10003a60 f   imageioJPEG.obj
 0001:00002a60       _Java_com_sun_imageio_plugins_jpeg_JPEGImageWriter_disposeWriter@16 10003a60 f   imageioJPEG.obj
 0001:00002ac0       _Java_com_sun_imageio_plugins_jpeg_JPEGImageWriter_initJPEGImageWriter@8 10003ac0 f   imageioJPEG.obj
 0001:00002c70       _JNI_OnLoad@8              10003c70 f   jpegdecoder.obj
 0001:00002db0       _sun_jpeg_fill_input_buffer 10003db0 f   jpegdecoder.obj
 0001:00002e90       _sun_jpeg_fill_suspended_buffer 10003e90 f   jpegdecoder.obj
 0001:00003020       _sun_jpeg_skip_input_data  10004020 f   jpegdecoder.obj
 0001:00003160       _Java_sun_awt_image_JPEGImageDecoder_initIDs@12 10004160 f   jpegdecoder.obj
 0001:000031f0       _Java_sun_awt_image_JPEGImageDecoder_readImage@16 100041f0 f   jpegdecoder.obj
 0001:00003650       _jAbort                    10004650 f   jcomapi.obj
 0001:00003690       _jDestroy                  10004690 f   jcomapi.obj
 0001:000036b0       _jAlcQTable                100046b0 f   jcomapi.obj
 0001:000036d0       _jAlcHTable                100046d0 f   jcomapi.obj
 0001:000036f0       _jCreaDecompress           100046f0 f   jdapimin.obj
 0001:000037e0       _jDestDecompress           100047e0 f   jdapimin.obj
 0001:000037f0       _jAbrtDecompress           100047f0 f   jdapimin.obj
 0001:00003990       _jConsumeInput             10004990 f   jdapimin.obj
 0001:00003a50       _jInComplete               10004a50 f   jdapimin.obj
 0001:00003aa0       _jHasMultScn               10004aa0 f   jdapimin.obj
 0001:00003af0       _jFinDecompress            10004af0 f   jdapimin.obj
 0001:00003bc0       _jReadHeader               10004bc0 f   jdapimin.obj
 0001:00003d00       _jReadScanlines            10004d00 f   jdapistd.obj
 0001:00003da0       _jStrtOutput               10004da0 f   jdapistd.obj
 0001:00003e10       _jFinOutput                10004e10 f   jdapistd.obj
 0001:00003eb0       _jStrtDecompress           10004eb0 f   jdapistd.obj
 0001:000042a0       _jMemInit                  100052a0 f   jmemnobs.obj
 0001:00004ec0       _jIDCoefC                  10005ec0 f   jdcoefct.obj
 0001:00005460       _jIDColor                  10006460 f   jdcolor.obj
 0001:00005960       _jIIDCT                    10006960 f   jddctmgr.obj
 0001:000059e0       _jMkDDerived               100069e0 f   jdhuff.obj
 0001:00005cb0       _jFilBitBuf                10006cb0 f   jdhuff.obj
 0001:00005de0       _jHufDecode                10006de0 f   jdhuff.obj
 0001:000064d0       _jIHDecoder                100074d0 f   jdhuff.obj
 0001:00006af0       _jIInCtlr                  10007af0 f   jdinput.obj
 0001:00007130       _jIDMainC                  10008130 f   jdmainct.obj
 0001:00008c80       _jResyncRestart            10009c80 f   jdmarker.obj
 0001:00008dc0       _jIMReader                 10009dc0 f   jdmarker.obj
 0001:00008e50       _jSaveMarkers              10009e50 f   jdmarker.obj
 0001:00008fa0       _jCalcDimensions           10009fa0 f   jdmaster.obj
 0001:000095b0       _jIDMaster                 1000a5b0 f   jdmaster.obj
 0001:00009b70       _jIMUpsampler              1000ab70 f   jdmerge.obj
 0001:0000a890       _jIPHDecoder               1000b890 f   jdphuff.obj
 0001:0000abc0       _jIDPostC                  1000bbc0 f   jdpostct.obj
 0001:0000b140       _jIUpsampler               1000c140 f   jdsample.obj
 0001:0000b4b0       _jStdError                 1000c4b0 f   jerror.obj
 0001:0000b500       _jRDfloat                  1000c500 f   jidctflt.obj
 0001:0000b930       _jRDifast                  1000c930 f   jidctfst.obj
 0001:0000bd20       _jRDislow                  1000cd20 f   jidctint.obj
 0001:0000c250       _jRD4x4                    1000d250 f   jidctred.obj
 0001:0000c570       _jRD2x2                    1000d570 f   jidctred.obj
 0001:0000c9e0       _jRD1x1                    1000d9e0 f   jidctred.obj
 0001:0000d530       _jIMemMgr                  1000e530 f   jmemmgr.obj
 0001:0000d660       _jGetLarge                 1000e660 f   jmemnobs.obj
 0001:0000d660       _jGetSmall                 1000e660 f   jmemnobs.obj
 0001:0000d670       _jFreeSmall                1000e670 f   jmemnobs.obj
 0001:0000d670       _jFreeLarge                1000e670 f   jmemnobs.obj
 0001:0000d680       _jMemAvail                 1000e680 f   jmemnobs.obj
 0001:0000d690       _jOpenBackStore            1000e690 f   jmemnobs.obj
 0001:0000d6b0       _jMemTerm                  1000e6b0 f   jmemnobs.obj
 0001:0000d6b0       _sun_jpeg_term_source      1000e6b0 f   jpegdecoder.obj
 0001:0000e240       _jI1Quant                  1000f240 f   jquant1.obj
 0001:0000f540       _jI2Quant                  10010540 f   jquant2.obj
 0001:0000f680       _jDivRound                 10010680 f   jutils.obj
 0001:0000f690       _jRound                    10010690 f   jutils.obj
 0001:0000f6b0       _jCopySamples              100106b0 f   jutils.obj
 0001:0000f700       _jCopyBlocks               10010700 f   jutils.obj
 0001:0000f730       _jZeroFar                  10010730 f   jutils.obj
 0001:0000f750       _jCreaCompress             10010750 f   jcapimin.obj
 0001:0000f820       _jSuppressTables           10010820 f   jcapimin.obj
 0001:0000f890       _jFinCompress              10010890 f   jcapimin.obj
 0001:0000f9a0       _jWrtTables                100109a0 f   jcapimin.obj
 0001:0000f9f0       _jStrtCompress             100109f0 f   jcapistd.obj
 0001:0000fa70       _jWrtScanlines             10010a70 f   jcapistd.obj
 0001:00010300       _jICCoefC                  10011300 f   jccoefct.obj
 0001:00010910       _jICColor                  10011910 f   jccolor.obj
 0001:00011900       _jIFDCT                    10012900 f   jcdctmgr.obj
 0001:00011990       _jMkCDerived               10012990 f   jchuff.obj
 0001:00012310       _jGenOptTbl                10013310 f   jchuff.obj
 0001:00012800       _jIHEncoder                10013800 f   jchuff.obj
 0001:00012860       _jICompress                10013860 f   jcinit.obj
 0001:00012a20       _jICMainC                  10013a20 f   jcmainct.obj
 0001:00013940       _jIMWriter                 10014940 f   jcmarker.obj
 0001:00014440       _jICMaster                 10015440 f   jcmaster.obj
 0001:00014500       _jAddQuantTable            10015500 f   jcparam.obj
 0001:000147f0       _jSetColorspace            100157f0 f   jcparam.obj
 0001:00014b40       _jSimProgress              10015b40 f   jcparam.obj
 0001:00014db0       _jDefColorspace            10015db0 f   jcparam.obj
 0001:00015060       _jSetDefaults              10016060 f   jcparam.obj
 0001:00015e50       _jIPHEncoder               10016e50 f   jcphuff.obj
 0001:00016450       _jICPrepC                  10017450 f   jcprepct.obj
 0001:00016d10       _jIDownsampler             10017d10 f   jcsample.obj
 0001:00016e90       _jFDfloat                  10017e90 f   jfdctflt.obj
 0001:00017fd0       _jFDifast                  10018fd0 f   jfdctfst.obj
 0001:000181e0       _jFDislow                  100191e0 f   jfdctint.obj
 0001:0001850e       _JNU_ThrowByName@12        1001950e f   java:java.dll
 0001:00018514       _JNU_GetEnv@8              10019514 f   java:java.dll
 0001:0001851a       _JNU_ThrowNullPointerException@8 1001951a f   java:java.dll
 0001:00018520       _jio_snprintf              10019520 f   java:java.dll
 0001:00018526       __setjmp3                  10019526 f   MSVCRT:MSVCR71.dll
 0001:00018530       __ftol2                    10019530 f   MSVCRT:ftol2.obj
 0001:000185a5       __CRT_INIT@12              100195a5 f   MSVCRT:crtdll.obj
 0001:00018663       __DllMainCRTStartup@12     10019663 f   MSVCRT:crtdll.obj
 0001:00018748       __initterm                 10019748 f   MSVCRT:MSVCR71.dll
 0001:0001874e       __onexit                   1001974e f   MSVCRT:atonexit.obj
 0001:00018774       _atexit                    10019774 f   MSVCRT:atonexit.obj
 0001:00018786       __RTC_Initialize           10019786 f   MSVCRT:initsect.obj
 0001:000187ca       __RTC_Terminate            100197ca f   MSVCRT:initsect.obj
 0001:0001880e       ___CppXcptFilter           1001980e f   MSVCRT:MSVCR71.dll
 0001:00018814       _DllMain@12                10019814 f   MSVCRT:dllmain.obj
 0001:00018834       __SEH_prolog               10019834 f   MSVCRT:sehprolg.obj
 0001:0001886f       __SEH_epilog               1001986f f   MSVCRT:sehprolg.obj
 0001:00018880       __except_handler3          10019880 f   MSVCRT:MSVCR71.dll
 0001:00018886       ___dllonexit               10019886 f   MSVCRT:MSVCR71.dll
 0002:00000000       __imp__DisableThreadLibraryCalls@4 1001a000     kernel32:KERNEL32.dll
 0002:00000004       \177KERNEL32_NULL_THUNK_DATA 1001a004     kernel32:KERNEL32.dll
 0002:00000008       __imp___onexit             1001a008     MSVCRT:MSVCR71.dll
 0002:0000000c       __imp____dllonexit         1001a00c     MSVCRT:MSVCR71.dll
 0002:00000010       __imp___assert             1001a010     MSVCRT:MSVCR71.dll
 0002:00000014       __imp__longjmp             1001a014     MSVCRT:MSVCR71.dll
 0002:00000018       __imp__free                1001a018     MSVCRT:MSVCR71.dll
 0002:0000001c       __imp___setjmp3            1001a01c     MSVCRT:MSVCR71.dll
 0002:00000020       __imp__malloc              1001a020     MSVCRT:MSVCR71.dll
 0002:00000024       __imp__fprintf             1001a024     MSVCRT:MSVCR71.dll
 0002:00000028       __imp___iob                1001a028     MSVCRT:MSVCR71.dll
 0002:0000002c       __imp__sscanf              1001a02c     MSVCRT:MSVCR71.dll
 0002:00000030       __imp__getenv              1001a030     MSVCRT:MSVCR71.dll
 0002:00000034       __imp___initterm           1001a034     MSVCRT:MSVCR71.dll
 0002:00000038       __imp___adjust_fdiv        1001a038     MSVCRT:MSVCR71.dll
 0002:0000003c       __imp____CppXcptFilter     1001a03c     MSVCRT:MSVCR71.dll
 0002:00000040       __imp___except_handler3    1001a040     MSVCRT:MSVCR71.dll
 0002:00000044       \177MSVCR71_NULL_THUNK_DATA 1001a044     MSVCRT:MSVCR71.dll
 0002:00000048       __imp__jio_snprintf        1001a048     java:java.dll
 0002:0000004c       __imp__JNU_ThrowNullPointerException@8 1001a04c     java:java.dll
 0002:00000050       __imp__JNU_GetEnv@8        1001a050     java:java.dll
 0002:00000054       __imp__JNU_ThrowByName@12  1001a054     java:java.dll
 0002:00000058       \177java_NULL_THUNK_DATA   1001a058     java:java.dll
 0002:0000007c       ??_C@_0BA@HDMLLOIA@sb?9?$DObuf?5?$DN?$DN?5NULL?$AA@ 1001a07c     imageioJPEG.obj
 0002:0000008c       ??_C@_0DL@MCJGNNBB@?4?4?1?4?4?1?4?4?1src?1share?1native?1sun?1aw@ 1001a08c     imageioJPEG.obj
 0002:000000c8       ??_C@_0BK@OBJDCLJJ@sb?9?$DOhstreamBuffer?5?$CB?$DN?5NULL?$AA@ 1001a0c8     imageioJPEG.obj
 0002:000000e4       ??_C@_0BL@ENCPOIKC@java?1lang?1OutOfMemoryError?$AA@ 1001a0e4     imageioJPEG.obj
 0002:00000100       ??_C@_0BF@GNONHPOP@Setting?5Pixel?5Buffer?$AA@ 1001a100     imageioJPEG.obj
 0002:00000118       ??_C@_0BD@DIGOHHHB@pb?9?$DObuf?4ip?5?$DN?$DN?5NULL?$AA@ 1001a118     imageioJPEG.obj
 0002:0000012c       ??_C@_0BJ@MKBLEEAK@pb?9?$DOhpixelObject?5?$CB?$DN?5NULL?$AA@ 1001a12c     imageioJPEG.obj
 0002:00000148       ??_C@_0CF@EJBMEBBP@Unable?5to?5pin?5icc?5profile?5data?5a@ 1001a148     imageioJPEG.obj
 0002:00000170       ??_C@_0BE@JBLDAGLI@Reading?5ICC?5profile?$AA@ 1001a170     imageioJPEG.obj
 0002:00000184       ??_C@_0CN@PIKPANEC@Invalid?5icc?5profile?3?5missing?5seq@ 1001a184     imageioJPEG.obj
 0002:000001b4       ??_C@_0CJ@PKIHEMMA@Invalid?5icc?5profile?3?5bad?5sequenc@ 1001a1b4     imageioJPEG.obj
 0002:000001e0       ??_C@_0DA@GLMLOKJH@Invalid?5icc?5profile?3?5duplicate?5s@ 1001a1e0     imageioJPEG.obj
 0002:00000210       ??_C@_0DF@EJNALACK@Invalid?5icc?5profile?3?5inconsisten@ 1001a210     imageioJPEG.obj
 0002:00000248       ??_C@_0BL@PAGFHBFL@javax?1imageio?1IIOException?$AA@ 1001a248     imageioJPEG.obj
 0002:00000264       ??_C@_0CO@ILDJFFGN@Invalid?5icc?5profile?3?5found?5only?5@ 1001a264     imageioJPEG.obj
 0002:00000294       ??_C@_06GEKOPAHD@values?$AA@ 1001a294     imageioJPEG.obj
 0002:0000029c       ??_C@_07HLHALEDB@lengths?$AA@ 1001a29c     imageioJPEG.obj
 0002:000002a4       ??_C@_02PBMBOJCL@?$FLS?$AA@ 1001a2a4     imageioJPEG.obj
 0002:000002a8       ??_C@_06NDKJHNCM@qTable?$AA@ 1001a2a8     imageioJPEG.obj
 0002:000002b0       ??_C@_02EBOMBDPA@?$FLI?$AA@ 1001a2b0     imageioJPEG.obj
 0002:000002b4       ??_C@_08FJPDKMKL@pushBack?$AA@ 1001a2b4     imageioJPEG.obj
 0002:000002c0       ??_C@_0N@JHOJIANF@passComplete?$AA@ 1001a2c0     imageioJPEG.obj
 0002:000002d0       ??_C@_03GAEACAIP@?$CI?$CJV?$AA@ 1001a2d0     imageioJPEG.obj
 0002:000002d4       ??_C@_0M@MNIOMPPJ@passStarted?$AA@ 1001a2d4     imageioJPEG.obj
 0002:000002e0       ??_C@_0N@NGMIGEIH@acceptPixels?$AA@ 1001a2e0     imageioJPEG.obj
 0002:000002f0       ??_C@_05IPOMILEE@?$CIIZ?$CJV?$AA@ 1001a2f0     imageioJPEG.obj
 0002:000002f8       ??_C@_0N@MNKCGBOF@setImageData?$AA@ 1001a2f8     imageioJPEG.obj
 0002:00000308       ??_C@_0L@NCAMOCKO@?$CIIIIII?$FLB?$CJV?$AA@ 1001a308     imageioJPEG.obj
 0002:00000314       ??_C@_0BD@EDGGINKI@warningWithMessage?$AA@ 1001a314     imageioJPEG.obj
 0002:00000328       ??_C@_0BG@IKDDPPGD@?$CILjava?1lang?1String?$DL?$CJV?$AA@ 1001a328     imageioJPEG.obj
 0002:00000340       ??_C@_0BA@CDPOJDB@warningOccurred?$AA@ 1001a340     imageioJPEG.obj
 0002:00000350       ??_C@_04PFANPMCN@?$CII?$CJV?$AA@ 1001a350     imageioJPEG.obj
 0002:00000358       ??_C@_0P@CHNKCPBH@skipInputBytes?$AA@ 1001a358     imageioJPEG.obj
 0002:00000368       ??_C@_04BMPAOJO@?$CIJ?$CJJ?$AA@ 1001a368     imageioJPEG.obj
 0002:00000370       ??_C@_0O@BACJPOFC@readInputData?$AA@ 1001a370     imageioJPEG.obj
 0002:00000380       ??_C@_07HGNEOLPD@?$CI?$FLBII?$CJI?$AA@ 1001a380     imageioJPEG.obj
 0002:00000388       ??_C@_0BB@BBPIIEJP@Array?5pin?5failed?$AA@ 1001a388     imageioJPEG.obj
 0002:0000039c       ??_C@_0CA@EJBFMCPI@java?1lang?1IllegalStateException?$AA@ 1001a39c     imageioJPEG.obj
 0002:000003bc       ??_C@_0CJ@FAHHFKDG@Attempting?5to?5use?5reader?5after?5d@ 1001a3bc     imageioJPEG.obj
 0002:000003e8       ??_C@_0CF@OPBCJGNA@Invalid?5argument?5to?5native?5readI@ 1001a3e8     imageioJPEG.obj
 0002:00000410       ??_C@_0CD@ODEKAMA@Invalid?5number?5of?5color?5componen@ 1001a410     imageioJPEG.obj
 0002:00000434       ??_C@_0BE@KOGPEOLP@Reading?5JPEG?5Stream?$AA@ 1001a434     imageioJPEG.obj
 0002:00000448       ??_C@_0BC@OMEGECOD@Initializing?5Read?$AA@ 1001a448     imageioJPEG.obj
 0002:0000045c       ??_C@_0BK@PBGJCCG@Output?5buffer?5not?5pinned?$CB?$AA@ 1001a45c     imageioJPEG.obj
 0002:00000478       ??_C@_0L@EKFGKJEH@grabPixels?$AA@ 1001a478     imageioJPEG.obj
 0002:00000484       ??_C@_0O@BLOPFHGH@writeMetadata?$AA@ 1001a484     imageioJPEG.obj
 0002:00000494       ??_C@_0BA@MONANPK@writeOutputData?$AA@ 1001a494     imageioJPEG.obj
 0002:000004a4       ??_C@_07LLIOOFGN@?$CI?$FLBII?$CJV?$AA@ 1001a4a4     imageioJPEG.obj
 0002:000004ac       ??_C@_0CJ@MCECMHCD@Attempting?5to?5use?5writer?5after?5d@ 1001a4ac     imageioJPEG.obj
 0002:000004d8       ??_C@_0CG@JKMPIIDL@Invalid?5argument?5to?5native?5write@ 1001a4d8     imageioJPEG.obj
 0002:00000500       ??_C@_0N@PEADDBOI@Writing?5JPEG?$AA@ 1001a500     imageioJPEG.obj
 0002:00000510       ??_C@_0BE@NMJJBJJA@Writing?5JPEG?5Stream?$AA@ 1001a510     imageioJPEG.obj
 0002:00000524       ??_C@_0O@FAOJELCO@Invalid?5Image?$AA@ 1001a524     imageioJPEG.obj
 0002:00000534       ??_C@_0P@FDFGJBFF@Setting?5Stream?$AA@ 1001a534     imageioJPEG.obj
 0002:00000544       ??_C@_0BE@LOJEHOGK@Initializing?5Reader?$AA@ 1001a544     imageioJPEG.obj
 0002:00000558       ??_C@_0BE@JCBGHPLA@Initializing?5Writer?$AA@ 1001a558     imageioJPEG.obj
 0002:0000056c       ??_C@_03OFAPEBGM@?$CFs?6?$AA@ 1001a56c     jpegdecoder.obj
 0002:00000570       ??_C@_0BE@DLILMMGE@src?9?$DOoutbuf?4ip?5?$DN?$DN?50?$AA@ 1001a570     jpegdecoder.obj
 0002:00000584       ??_C@_0BA@JDGFEGAG@src?9?$DOinbuf?5?$DN?$DN?50?$AA@ 1001a584     jpegdecoder.obj
 0002:00000594       ??_C@_0DL@BENJPMGD@?4?4?1?4?4?1?4?4?1src?1share?1native?1sun?1aw@ 1001a594     jpegdecoder.obj
 0002:000005d0       ??_C@_09LAIKOIHJ@available?$AA@ 1001a5d0     jpegdecoder.obj
 0002:000005dc       ??_C@_03KNBKCOBB@?$CI?$CJI?$AA@ 1001a5dc     jpegdecoder.obj
 0002:000005e0       ??_C@_04POLDLDMI@read?$AA@ 1001a5e0     jpegdecoder.obj
 0002:000005e8       ??_C@_06DMLPEKHA@?$CI?$FLII?$CJZ?$AA@ 1001a5e8     jpegdecoder.obj
 0002:000005f0       ??_C@_0L@IINNECMJ@sendPixels?$AA@ 1001a5f0     jpegdecoder.obj
 0002:000005fc       ??_C@_06ELGPHLGB@?$CI?$FLBI?$CJZ?$AA@ 1001a5fc     jpegdecoder.obj
 0002:00000604       ??_C@_0P@BDIPJFFC@sendHeaderInfo?$AA@ 1001a604     jpegdecoder.obj
 0002:00000614       ??_C@_08MLFAPJAK@?$CIIIZZZ?$CJZ?$AA@ 1001a614     jpegdecoder.obj
 0002:00000620       ??_C@_0CD@OMFLCCFG@sun?1awt?1image?1ImageFormatExcepti@ 1001a620     jpegdecoder.obj
 0002:00000648       __real@3ff0000000000000    1001a648     jdapimin.obj
 0002:00000710       __real@3fd1a855de72ab5d    1001a710     jddctmgr.obj
 0002:00000718       __real@3fe1517a7bc720bb    1001a718     jddctmgr.obj
 0002:00000720       __real@3fe92469c0a7bf3b    1001a720     jddctmgr.obj
 0002:00000728       __real@3ff2d062ef6c11aa    1001a728     jddctmgr.obj
 0002:00000730       __real@3ff4e7ae914d6fca    1001a730     jddctmgr.obj
 0002:00000738       __real@3ff63150b14861ef    1001a738     jddctmgr.obj
 0002:00000840       _jMsgTable                 1001a840     jerror.obj
 0002:00000a34       ??_C@_0CL@OCGBAKPF@Application?5transferred?5too?5many@ 1001aa34     jerror.obj
 0002:00000a60       ??_C@_0CL@BAKCGOKJ@Invalid?5SOS?5parameters?5for?5seque@ 1001aa60     jerror.obj
 0002:00000a8c       ??_C@_0DI@NFMBADOH@Corrupt?5JPEG?5data?3?5found?5marker?5@ 1001aa8c     jerror.obj
 0002:00000ac4       ??_C@_0BL@DPFPFMLM@Premature?5end?5of?5JPEG?5file?$AA@ 1001aac4     jerror.obj
 0002:00000ae0       ??_C@_0CO@ODCCEDLN@Warning?3?5unknown?5JFIF?5revision?5n@ 1001aae0     jerror.obj
 0002:00000b10       ??_C@_0CE@PBLDOPKB@Corrupt?5JPEG?5data?3?5bad?5Huffman?5c@ 1001ab10     jerror.obj
 0002:00000b34       ??_C@_0DB@PGMEPGHN@Corrupt?5JPEG?5data?3?5premature?5end@ 1001ab34     jerror.obj
 0002:00000b68       ??_C@_0DM@PCOGCKJB@Corrupt?5JPEG?5data?3?5?$CFu?5extraneous@ 1001ab68     jerror.obj
 0002:00000ba8       ??_C@_0EC@CBCJOINE@Inconsistent?5progression?5sequenc@ 1001aba8     jerror.obj
 0002:00000bec       ??_C@_0CG@KEGHCDOM@Unknown?5Adobe?5color?5transform?5co@ 1001abec     jerror.obj
 0002:00000c14       ??_C@_0BH@LJLGPEFF@Obtained?5XMS?5handle?5?$CFu?$AA@ 1001ac14     jerror.obj
 0002:00000c2c       ??_C@_0BE@FOGGKKAO@Freed?5XMS?5handle?5?$CFu?$AA@ 1001ac2c     jerror.obj
 0002:00000c40       ??_C@_0DE@EEJCDLOO@Unrecognized?5component?5IDs?5?$CFd?5?$CFd@ 1001ac40     jerror.obj
 0002:00000c74       ??_C@_0DG@FCFDGNHE@JFIF?5extension?5marker?3?5RGB?5thumb@ 1001ac74     jerror.obj
 0002:00000cac       ??_C@_0DK@JGAPDCJL@JFIF?5extension?5marker?3?5palette?5t@ 1001acac     jerror.obj
 0002:00000ce8       ??_C@_0EC@ELDEPOJP@JFIF?5extension?5marker?3?5JPEG?9comp@ 1001ace8     jerror.obj
 0002:00000d2c       ??_C@_0BJ@GOCABEP@Opened?5temporary?5file?5?$CFs?$AA@ 1001ad2c     jerror.obj
 0002:00000d48       ??_C@_0BJ@KDCGAOJB@Closed?5temporary?5file?5?$CFs?$AA@ 1001ad48     jerror.obj
 0002:00000d64       ??_C@_0BN@GAMIJLDC@?5?5Ss?$DN?$CFd?0?5Se?$DN?$CFd?0?5Ah?$DN?$CFd?0?5Al?$DN?$CFd?$AA@ 1001ad64     jerror.obj
 0002:00000d84       ??_C@_0BO@CDEKFGLC@?5?5?5?5Component?5?$CFd?3?5dc?$DN?$CFd?5ac?$DN?$CFd?$AA@ 1001ad84     jerror.obj
 0002:00000da4       ??_C@_0BN@BLOOHNC@Start?5Of?5Scan?3?5?$CFd?5components?$AA@ 1001ada4     jerror.obj
 0002:00000dc4       ??_C@_0P@JLCHJELA@Start?5of?5Image?$AA@ 1001adc4     jerror.obj
 0002:00000dd4       ??_C@_0BP@EDCAMHHE@?5?5?5?5Component?5?$CFd?3?5?$CFdhx?$CFdv?5q?$DN?$CFd?$AA@ 1001add4     jerror.obj
 0002:00000df4       ??_C@_0DK@DMINKOGN@Start?5Of?5Frame?50x?$CF02x?3?5width?$DN?$CFu?0@ 1001adf4     jerror.obj
 0002:00000e30       ??_C@_0DJ@PCBCLFML@Smoothing?5not?5supported?5with?5non@ 1001ae30     jerror.obj
 0002:00000e6c       ??_C@_05LLAPAOG@RST?$CFd?$AA@ 1001ae6c     jerror.obj
 0002:00000e74       ??_C@_0CF@NIMOLBCP@At?5marker?50x?$CF02x?0?5recovery?5actio@ 1001ae74     jerror.obj
 0002:00000e9c       ??_C@_0CE@FDPBEAOO@Selected?5?$CFd?5colors?5for?5quantizat@ 1001ae9c     jerror.obj
 0002:00000ec0       ??_C@_0BI@NEIBNACE@Quantizing?5to?5?$CFd?5colors?$AA@ 1001aec0     jerror.obj
 0002:00000ed8       ??_C@_0CD@CNNAOOFA@Quantizing?5to?5?$CFd?5?$DN?5?$CFd?$CK?$CFd?$CK?$CFd?5colo@ 1001aed8     jerror.obj
 0002:00000efc       ??_C@_0CI@GHPOCOCL@?5?5?5?5?5?5?5?5?$CF4u?5?$CF4u?5?$CF4u?5?$CF4u?5?$CF4u?5?$CF4u?5@ 1001aefc     jerror.obj
 0002:00000f24       ??_C@_0BJ@COPODLDN@Unexpected?5marker?50x?$CF02x?$AA@ 1001af24     jerror.obj
 0002:00000f40       ??_C@_0CH@EHHJCMGA@Miscellaneous?5marker?50x?$CF02x?0?5len@ 1001af40     jerror.obj
 0002:00000f68       ??_C@_0CB@BADBMAAB@?5?5?5?5with?5?$CFd?5x?5?$CFd?5thumbnail?5image@ 1001af68     jerror.obj
 0002:00000f8c       ??_C@_0CO@KKPHGHBA@JFIF?5extension?5marker?3?5type?50x?$CF0@ 1001af8c     jerror.obj
 0002:00000fbc       ??_C@_0DM@JLHNPIBE@Warning?3?5thumbnail?5image?5size?5do@ 1001afbc     jerror.obj
 0002:00000ff8       ??_C@_0DF@LOKNABIG@JFIF?5APP0?5marker?3?5version?5?$CFd?4?$CF02@ 1001aff8     jerror.obj
 0002:00001030       ??_C@_0CI@FKGPAJC@?5?5?5?5?5?5?5?5?$CF3d?5?$CF3d?5?$CF3d?5?$CF3d?5?$CF3d?5?$CF3d?5@ 1001b030     jerror.obj
 0002:00001058       ??_C@_0N@HJHFKELG@End?5Of?5Image?$AA@ 1001b058     jerror.obj
 0002:00001068       ??_C@_0BH@GIPOLIGC@Obtained?5EMS?5handle?5?$CFu?$AA@ 1001b068     jerror.obj
 0002:00001080       ??_C@_0BE@IPCOOGDJ@Freed?5EMS?5handle?5?$CFu?$AA@ 1001b080     jerror.obj
 0002:00001094       ??_C@_0BL@EMFIKBEK@Define?5Restart?5Interval?5?$CFu?$AA@ 1001b094     jerror.obj
 0002:000010b0       ??_C@_0CL@KLDOJIKN@Define?5Quantization?5Table?5?$CFd?5?5pr@ 1001b0b0     jerror.obj
 0002:000010dc       ??_C@_0BM@MDIEILCE@Define?5Huffman?5Table?50x?$CF02x?$AA@ 1001b0dc     jerror.obj
 0002:000010f8       ??_C@_0CH@KIJGKPAA@Define?5Arithmetic?5Table?50x?$CF02x?3?5@ 1001b0f8     jerror.obj
 0002:00001120       ??_C@_0CM@CAEPHFAA@Unknown?5APP14?5marker?5?$CInot?5Adobe?$CJ@ 1001b120     jerror.obj
 0002:0000114c       ??_C@_0CK@HCPFFNKJ@Unknown?5APP0?5marker?5?$CInot?5JFIF?$CJ?0?5@ 1001b14c     jerror.obj
 0002:00001178       ??_C@_0EC@EHPKAOHA@Adobe?5APP14?5marker?3?5version?5?$CFd?0?5@ 1001b178     jerror.obj
 0002:000011bc       ??_C@_0DO@EGLODMBB@Caution?3?5quantization?5tables?5are@ 1001b1bc     jerror.obj
 0002:000011fc       ??_C@_0BA@LIJBPGPA@6b?5?527?9Mar?91998?$AA@ 1001b1fc     jerror.obj
 0002:0000120c       ??_C@_0CD@IMBKIDCD@Copyright?5?$CIC?$CJ?51998?0?5Thomas?5G?4?5La@ 1001b20c     jerror.obj
 0002:00001230       ??_C@_0BE@FDPDCBIN@Write?5to?5XMS?5failed?$AA@ 1001b230     jerror.obj
 0002:00001244       ??_C@_0BF@EKLGFGNM@Read?5from?5XMS?5failed?$AA@ 1001b244     jerror.obj
 0002:0000125c       ??_C@_0CH@LJLHCCHC@Image?5too?5wide?5for?5this?5implemen@ 1001b25c     jerror.obj
 0002:00001284       ??_C@_0CD@GCLFJCHC@Virtual?5array?5controller?5messed?5@ 1001b284     jerror.obj
 0002:000012a8       ??_C@_0BP@BPKOBOIP@Unsupported?5marker?5type?50x?$CF02x?$AA@ 1001b2a8     jerror.obj
 0002:000012c8       ??_C@_0CK@EPADOAKC@Application?5transferred?5too?5few?5@ 1001b2c8     jerror.obj
 0002:000012f4       ??_C@_0DG@KALDLIJB@Write?5failed?5on?5temporary?5file?5?9@ 1001b2f4     jerror.obj
 0002:0000132c       ??_C@_0BO@GOBJOAAI@Seek?5failed?5on?5temporary?5file?$AA@ 1001b32c     jerror.obj
 0002:0000134c       ??_C@_0BO@EEPJGHHI@Read?5failed?5on?5temporary?5file?$AA@ 1001b34c     jerror.obj
 0002:0000136c       ??_C@_0CD@POKNOPOF@Failed?5to?5create?5temporary?5file?5@ 1001b36c     jerror.obj
 0002:00001390       ??_C@_0CM@HONLBDPH@Invalid?5JPEG?5file?5structure?3?5SOS@ 1001b390     jerror.obj
 0002:000013bc       ??_C@_0CN@HGJCMLNE@Invalid?5JPEG?5file?5structure?3?5two@ 1001b3bc     jerror.obj
 0002:000013ec       ??_C@_0CK@HMKECJK@Unsupported?5JPEG?5process?3?5SOF?5ty@ 1001b3ec     jerror.obj
 0002:00001418       ??_C@_0DA@GJIJGINK@Invalid?5JPEG?5file?5structure?3?5mis@ 1001b418     jerror.obj
 0002:00001448       ??_C@_0CN@IHJJJAFJ@Invalid?5JPEG?5file?5structure?3?5two@ 1001b448     jerror.obj
 0002:00001478       ??_C@_0CH@NHMNHHIB@Cannot?5quantize?5to?5more?5than?5?$CFd?5@ 1001b478     jerror.obj
 0002:000014a0       ??_C@_0CI@PLMPLCNO@Cannot?5quantize?5to?5fewer?5than?5?$CFd@ 1001b4a0     jerror.obj
 0002:000014c8       ??_C@_0CO@HPDBAEEA@Cannot?5quantize?5more?5than?5?$CFd?5col@ 1001b4c8     jerror.obj
 0002:000014f8       ??_C@_0BO@DJPLELIB@Insufficient?5memory?5?$CIcase?5?$CFd?$CJ?$AA@ 1001b4f8     jerror.obj
 0002:00001518       ??_C@_0CL@GNLFDFCL@Not?5a?5JPEG?5file?3?5starts?5with?50x?$CF@ 1001b518     jerror.obj
 0002:00001544       ??_C@_0CK@CCHKIENB@Quantization?5table?50x?$CF02x?5was?5no@ 1001b544     jerror.obj
 0002:00001570       ??_C@_0CC@BKPLBDLJ@JPEG?5datastream?5contains?5no?5imag@ 1001b570     jerror.obj
 0002:00001594       ??_C@_0CF@BKANFCCL@Huffman?5table?50x?$CF02x?5was?5not?5def@ 1001b594     jerror.obj
 0002:000015bc       ??_C@_0BM@HJHFKLAF@Backing?5store?5not?5supported?$AA@ 1001b5bc     jerror.obj
 0002:000015d8       ??_C@_0CO@BEHINNOI@Requested?5feature?5was?5omitted?5at@ 1001b5d8     jerror.obj
 0002:00001608       ??_C@_0BE@EOAAHHJ@Not?5implemented?5yet?$AA@ 1001b608     jerror.obj
 0002:0000161c       ??_C@_0CH@EFBBPPCK@Invalid?5color?5quantization?5mode?5@ 1001b61c     jerror.obj
 0002:00001644       ??_C@_0CH@NIBDNILP@Scan?5script?5does?5not?5transmit?5al@ 1001b644     jerror.obj
 0002:0000166c       ??_C@_0DO@OPNPKGO@Cannot?5transcode?5due?5to?5multiple@ 1001b66c     jerror.obj
 0002:000016ac       ??_C@_0BM@KEKMMNGA@Premature?5end?5of?5input?5file?$AA@ 1001b6ac     jerror.obj
 0002:000016c8       ??_C@_0BB@JJAIKFBB@Empty?5input?5file?$AA@ 1001b6c8     jerror.obj
 0002:000016dc       ??_C@_0CP@EKFPGPNP@Maximum?5supported?5image?5dimensio@ 1001b6dc     jerror.obj
 0002:0000170c       ??_C@_0CB@LFBMFPHI@Missing?5Huffman?5code?5table?5entry@ 1001b70c     jerror.obj
 0002:00001730       ??_C@_0CB@LLDOGNPJ@Huffman?5code?5size?5table?5overflow@ 1001b730     jerror.obj
 0002:00001754       ??_C@_0CI@EKDDDHFF@Fractional?5sampling?5not?5implemen@ 1001b754     jerror.obj
 0002:0000177c       ??_C@_0CP@IDOBLGGD@Output?5file?5write?5error?5?9?9?9?5out?5@ 1001b77c     jerror.obj
 0002:000017ac       ??_C@_0BG@BALCKDNL@Input?5file?5read?5error?$AA@ 1001b7ac     jerror.obj
 0002:000017c4       ??_C@_0CB@DMGINPNE@Didn?8t?5expect?5more?5than?5one?5scan@ 1001b7c4     jerror.obj
 0002:000017e8       ??_C@_0BE@DGJBKIEB@Write?5to?5EMS?5failed?$AA@ 1001b7e8     jerror.obj
 0002:000017fc       ??_C@_0BF@CPNENPBA@Read?5from?5EMS?5failed?$AA@ 1001b7fc     jerror.obj
 0002:00001814       ??_C@_0CF@DAGGEAPM@Empty?5JPEG?5image?5?$CIDNL?5not?5suppor@ 1001b814     jerror.obj
 0002:0000183c       ??_C@_0BD@DIMECAOP@Bogus?5DQT?5index?5?$CFd?$AA@ 1001b83c     jerror.obj
 0002:00001850       ??_C@_0BD@KJHFPHIC@Bogus?5DHT?5index?5?$CFd?$AA@ 1001b850     jerror.obj
 0002:00001864       ??_C@_0BF@CLIOOJFM@Bogus?5DAC?5value?50x?$CFx?$AA@ 1001b864     jerror.obj
 0002:0000187c       ??_C@_0BD@LDBBBMFL@Bogus?5DAC?5index?5?$CFd?$AA@ 1001b87c     jerror.obj
 0002:00001890       ??_C@_0CF@JDLOPNGO@Unsupported?5color?5conversion?5req@ 1001b890     jerror.obj
 0002:000018b8       ??_C@_0CG@BEBDNOCG@Too?5many?5color?5components?3?5?$CFd?0?5m@ 1001b8b8     jerror.obj
 0002:000018e0       ??_C@_0CF@LAEFHNAH@CCIR601?5sampling?5not?5implemented@ 1001b8e0     jerror.obj
 0002:00001908       ??_C@_0BM@PKHCPJDH@Suspension?5not?5allowed?5here?$AA@ 1001b908     jerror.obj
 0002:00001924       ??_C@_0CL@JKHIPJLJ@Buffer?5passed?5to?5JPEG?5library?5is@ 1001b924     jerror.obj
 0002:00001950       ??_C@_0BL@CBOEEPLK@Bogus?5virtual?5array?5access?$AA@ 1001b950     jerror.obj
 0002:00001970       ??_C@_0EN@DKAEGIBH@JPEG?5parameter?5struct?5mismatch?3?5@ 1001b970     jerror.obj
 0002:000019c0       ??_C@_0CK@BAMFIBMM@Improper?5call?5to?5JPEG?5library?5in@ 1001b9c0     jerror.obj
 0002:000019ec       ??_C@_0CA@MJDDICLK@Invalid?5scan?5script?5at?5entry?5?$CFd?$AA@ 1001b9ec     jerror.obj
 0002:00001a0c       ??_C@_0BH@HMMHPOPE@Bogus?5sampling?5factors?$AA@ 1001ba0c     jerror.obj
 0002:00001a24       ??_C@_0DH@HIKEGPKP@Invalid?5progressive?5parameters?5a@ 1001ba24     jerror.obj
 0002:00001a5c       ??_C@_0DH@LNGGEGOL@Invalid?5progressive?5parameters?5S@ 1001ba5c     jerror.obj
 0002:00001a94       ??_C@_0CD@LDBDNLHK@Unsupported?5JPEG?5data?5precision?5@ 1001ba94     jerror.obj
 0002:00001ab8       ??_C@_0BM@OEMICEFD@Invalid?5memory?5pool?5code?5?$CFd?$AA@ 1001bab8     jerror.obj
 0002:00001ad4       ??_C@_0DA@HLEOHNPA@Sampling?5factors?5too?5large?5for?5i@ 1001bad4     jerror.obj
 0002:00001b04       ??_C@_0DN@ELFKFKL@Wrong?5JPEG?5library?5version?3?5libr@ 1001bb04     jerror.obj
 0002:00001b44       ??_C@_0BE@OGLAEMOG@Bogus?5marker?5length?$AA@ 1001bb44     jerror.obj
 0002:00001b58       ??_C@_0BG@NEGIHEMC@Bogus?5JPEG?5colorspace?$AA@ 1001bb58     jerror.obj
 0002:00001b70       ??_C@_0BH@BGDIGLHC@Bogus?5input?5colorspace?$AA@ 1001bb70     jerror.obj
 0002:00001b88       ??_C@_0BP@EOFJNLFD@Bogus?5Huffman?5table?5definition?$AA@ 1001bb88     jerror.obj
 0002:00001ba8       ??_C@_0CI@MBJANLAP@IDCT?5output?5block?5size?5?$CFd?5not?5su@ 1001bba8     jerror.obj
 0002:00001bd0       ??_C@_0BN@OJEJKKDL@DCT?5coefficient?5out?5of?5range?$AA@ 1001bbd0     jerror.obj
 0002:00001bf0       ??_C@_0BP@ONFLCDHG@Invalid?5component?5ID?5?$CFd?5in?5SOS?$AA@ 1001bbf0     jerror.obj
 0002:00001c10       ??_C@_0BK@DKALDNKG@Bogus?5buffer?5control?5mode?$AA@ 1001bc10     jerror.obj
 0002:00001c2c       ??_C@_0CF@DENLILGA@MAX_ALLOC_CHUNK?5is?5wrong?0?5please@ 1001bc2c     jerror.obj
 0002:00001c54       ??_C@_0CA@FDMPGPNI@ALIGN_TYPE?5is?5wrong?0?5please?5fix?$AA@ 1001bc54     jerror.obj
 0002:00001c74       ??_C@_0DJ@KONAFFHE@Sorry?0?5there?5are?5legal?5restricti@ 1001bc74     jerror.obj
 0002:00001cb0       ??_C@_0BG@MIBALFBH@Bogus?5message?5code?5?$CFd?$AA@ 1001bcb0     jerror.obj
 0002:00001cc8       __real@3f8a8bd4            1001bcc8     jidctflt.obj
 0002:00001ccc       __real@40273d75            1001bccc     jidctflt.obj
 0002:00001cd0       __real@3fec835e            1001bcd0     jidctflt.obj
 0002:00001cd4       __real@3fb504f3            1001bcd4     jidctflt.obj
 0002:00001ce8       ??_C@_05IBIMIMKO@?$CFld?$CFc?$AA@ 1001bce8     jmemmgr.obj
 0002:00001cf0       ??_C@_07OOOLPGAB@JPEGMEM?$AA@ 1001bcf0     jmemmgr.obj
 0002:00001e08       _jZAGTable                 1001be08     jutils.obj
 0002:00002008       __real@4001a855de72ab5d    1001c008     jcdctmgr.obj
 0002:00002010       __real@4011517a7bc720bb    1001c010     jcdctmgr.obj
 0002:00002018       __real@40192469c0a7bf3b    1001c018     jcdctmgr.obj
 0002:00002020       __real@4022d062ef6c11aa    1001c020     jcdctmgr.obj
 0002:00002028       __real@4024e7ae914d6fca    1001c028     jcdctmgr.obj
 0002:00002030       __real@40263150b14861ef    1001c030     jcdctmgr.obj
 0002:00002038       __real@4020000000000000    1001c038     jcdctmgr.obj
 0002:00002040       __real@46800100            1001c040     jcdctmgr.obj
 0002:000023fc       __real@3fa73d75            1001c3fc     jfdctflt.obj
 0002:00002400       __real@3f0a8bd4            1001c400     jfdctflt.obj
 0002:00002404       __real@3ec3ef15            1001c404     jfdctflt.obj
 0002:00002408       __real@3f3504f3            1001c408     jfdctflt.obj
 0002:00002440       __load_config_used         1001c440     MSVCRT:loadcfg.obj
 0002:000024e0       ___safe_se_handler_table   1001c4e0     <linker-defined>
 0002:000024e4       ___rtc_iaa                 1001c4e4     MSVCRT:initsect.obj
 0002:000024e8       ___rtc_izz                 1001c4e8     MSVCRT:initsect.obj
 0002:000024ec       ___rtc_taa                 1001c4ec     MSVCRT:initsect.obj
 0002:000024f0       ___rtc_tzz                 1001c4f0     MSVCRT:initsect.obj
 0002:000024f4       __IMPORT_DESCRIPTOR_java   1001c4f4     java:java.dll
 0002:00002508       __IMPORT_DESCRIPTOR_MSVCR71 1001c508     MSVCRT:MSVCR71.dll
 0002:0000251c       __IMPORT_DESCRIPTOR_KERNEL32 1001c51c     kernel32:KERNEL32.dll
 0002:00002530       __NULL_IMPORT_DESCRIPTOR   1001c530     java:java.dll
 0003:00000000       ___xc_a                    1001d000     MSVCRT:cinitexe.obj
 0003:00000004       ___xc_z                    1001d004     MSVCRT:cinitexe.obj
 0003:00000008       ___xi_a                    1001d008     MSVCRT:cinitexe.obj
 0003:0000000c       ___xi_z                    1001d00c     MSVCRT:cinitexe.obj
 0003:00000010       ___security_cookie         1001d010     MSVCRT:seccook.obj
 0003:00000070       _jvm                       1001d070     <common>
 0003:00000074       __adjust_fdiv              1001d074     <common>
 0003:00000078       ___onexitend               1001d078     <common>
 0003:0000007c       ___onexitbegin             1001d07c     <common>
 0003:00000080       __pRawDllMain              1001d080     <common>

 entry point at        0001:00018663

 Static symbols

 0001:00000000       _pinStreamBuffer           10001000 f   imageioJPEG.obj
 0001:00000060       _unpinStreamBuffer         10001060 f   imageioJPEG.obj
 0001:000000c0       _setPixelBuffer            100010c0 f   imageioJPEG.obj
 0001:00000100       _RELEASE_ARRAYS            10001100 f   imageioJPEG.obj
 0001:00000150       _GET_ARRAYS                10001150 f   imageioJPEG.obj
 0001:000001c0       _sun_jpeg_output_message   100011c0 f   imageioJPEG.obj
 0001:00000230       _setQTables                10001230 f   imageioJPEG.obj
 0001:00000330       _setHuffTable              10001330 f   imageioJPEG.obj
 0001:00000410       _setHTables                10001410 f   imageioJPEG.obj
 0001:00001760       _imageio_init_destination  10002760 f   imageioJPEG.obj
 0001:000017a0       _imageio_empty_output_buffer 100027a0 f   imageioJPEG.obj
 0001:00001880       _imageio_term_destination  10002880 f   imageioJPEG.obj
 0001:00001910       _imageio_flush_destination 10002910 f   imageioJPEG.obj
 0001:000023c0       _resetStreamBuffer         100033c0 f   imageioJPEG.obj
 0001:00002430       _imageio_set_stream        10003430 f   imageioJPEG.obj
 0001:000024f0       _imageio_reset             100034f0 f   imageioJPEG.obj
 0001:00002730       _initStreamBuffer          10003730 f   imageioJPEG.obj
 0001:000027a0       _initImageioData           100037a0 f   imageioJPEG.obj
 0001:00002850       _destroyImageioData        10003850 f   imageioJPEG.obj
 0001:00002c90       _sun_jpeg_error_exit       10003c90 f   jpegdecoder.obj
 0001:00002c90       _sun_jpeg_error_exit       10003c90 f   jpegdecoder.obj
 0001:00002cb0       _RELEASE_ARRAYS            10003cb0 f   jpegdecoder.obj
 0001:00002d10       _GET_ARRAYS                10003d10 f   jpegdecoder.obj
 0001:00003800       _default_decompress_parms  10004800 f   jdapimin.obj
 0001:00003c30       _output_pass_setup         10004c30 f   jdapistd.obj
 0001:00003f90       _start_iMCU_row            10004f90 f   jdcoefct.obj
 0001:00003fe0       _start_input_pass          10004fe0 f   jdcoefct.obj
 0001:00004000       _decompress_onepass        10005000 f   jdcoefct.obj
 0001:000042a0       _dummy_consume_data        100052a0 f   jdcoefct.obj
 0001:000042b0       _consume_data              100052b0 f   jdcoefct.obj
 0001:000044e0       _decompress_data           100054e0 f   jdcoefct.obj
 0001:00004690       _smoothing_ok              10005690 f   jdcoefct.obj
 0001:00004800       _decompress_smooth_data    10005800 f   jdcoefct.obj
 0001:00004e70       _start_output_pass         10005e70 f   jdcoefct.obj
 0001:00005010       _build_ycc_rgb_table       10006010 f   jdcolor.obj
 0001:000050e0       _ycc_rgb_convert           100060e0 f   jdcolor.obj
 0001:00005200       _null_convert              10006200 f   jdcolor.obj
 0001:00005280       _grayscale_convert         10006280 f   jdcolor.obj
 0001:000052b0       _gray_rgb_convert          100062b0 f   jdcolor.obj
 0001:00005310       _ycck_cmyk_convert         10006310 f   jdcolor.obj
 0001:00005630       _start_pass                10006630 f   jddctmgr.obj
 0001:00005ec0       _process_restart           10006ec0 f   jdhuff.obj
 0001:00005f50       _decode_mcu                10006f50 f   jdhuff.obj
 0001:00006370       _start_pass_huff_decoder   10007370 f   jdhuff.obj
 0001:00006520       _initial_setup             10007520 f   jdinput.obj
 0001:00006720       _per_scan_setup            10007720 f   jdinput.obj
 0001:000068c0       _latch_quant_tables        100078c0 f   jdinput.obj
 0001:00006970       _start_input_pass          10007970 f   jdinput.obj
 0001:000069b0       _consume_markers           100079b0 f   jdinput.obj
 0001:00006a80       _reset_input_controller    10007a80 f   jdinput.obj
 0001:00006ad0       _finish_input_pass         10007ad0 f   jdinput.obj
 0001:00006b40       _alloc_funny_pointers      10007b40 f   jdmainct.obj
 0001:00006bf0       _make_funny_pointers       10007bf0 f   jdmainct.obj
 0001:00006d40       _set_wraparound_pointers   10007d40 f   jdmainct.obj
 0001:00006e20       _set_bottom_pointers       10007e20 f   jdmainct.obj
 0001:00006ec0       _process_data_simple_main  10007ec0 f   jdmainct.obj
 0001:00006f40       _process_data_context_main 10007f40 f   jdmainct.obj
 0001:00007080       _process_data_crank_post   10008080 f   jdmainct.obj
 0001:000070b0       _start_pass_main           100080b0 f   jdmainct.obj
 0001:00007200       _get_soi                   10008200 f   jdmarker.obj
 0001:000072b0       _get_sof                   100082b0 f   jdmarker.obj
 0001:000075d0       _get_sos                   100085d0 f   jdmarker.obj
 0001:00007920       _get_dht                   10008920 f   jdmarker.obj
 0001:00007c30       _get_dqt                   10008c30 f   jdmarker.obj
 0001:00007e90       _get_dri                   10008e90 f   jdmarker.obj
 0001:00007f80       _examine_app0              10008f80 f   jdmarker.obj
 0001:000081d0       _examine_app14             100091d0 f   jdmarker.obj
 0001:00008280       _get_interesting_appn      10009280 f   jdmarker.obj
 0001:000083d0       _save_marker               100093d0 f   jdmarker.obj
 0001:00008650       _skip_variable             10009650 f   jdmarker.obj
 0001:000086f0       _next_marker               100096f0 f   jdmarker.obj
 0001:00008800       _first_marker              10009800 f   jdmarker.obj
 0001:000088a0       _read_markers              100098a0 f   jdmarker.obj
 0001:00008bf0       _read_restart_marker       10009bf0 f   jdmarker.obj
 0001:00008d90       _reset_marker_reader       10009d90 f   jdmarker.obj
 0001:00008f20       _use_merged_upsample       10009f20 f   jdmaster.obj
 0001:000091d0       _prepare_range_limit_table 1000a1d0 f   jdmaster.obj
 0001:00009250       _master_selection          1000a250 f   jdmaster.obj
 0001:00009420       _prepare_for_output_pass   1000a420 f   jdmaster.obj
 0001:00009580       _finish_output_pass        1000a580 f   jdmaster.obj
 0001:000095f0       _build_ycc_rgb_table       1000a5f0 f   jdmerge.obj
 0001:000096c0       _start_pass_merged_upsample 1000a6c0 f   jdmerge.obj
 0001:000096e0       _merged_2v_upsample        1000a6e0 f   jdmerge.obj
 0001:000097b0       _merged_1v_upsample        1000a7b0 f   jdmerge.obj
 0001:000097f0       _h2v1_merged_upsample      1000a7f0 f   jdmerge.obj
 0001:00009940       _h2v2_merged_upsample      1000a940 f   jdmerge.obj
 0001:00009bf0       _process_restart           1000abf0 f   jdphuff.obj
 0001:00009c80       _decode_mcu_DC_first       1000ac80 f   jdphuff.obj
 0001:00009ed0       _decode_mcu_AC_first       1000aed0 f   jdphuff.obj
 0001:0000a120       _decode_mcu_DC_refine      1000b120 f   jdphuff.obj
 0001:0000a210       _decode_mcu_AC_refine      1000b210 f   jdphuff.obj
 0001:0000a610       _start_pass_phuff_decoder  1000b610 f   jdphuff.obj
 0001:0000a900       _post_process_1pass        1000b900 f   jdpostct.obj
 0001:0000a980       _post_process_prepass      1000b980 f   jdpostct.obj
 0001:0000aa20       _post_process_2pass        1000ba20 f   jdpostct.obj
 0001:0000aac0       _start_pass_dpost          1000bac0 f   jdpostct.obj
 0001:0000ac50       _start_pass_upsample       1000bc50 f   jdsample.obj
 0001:0000ac70       _sep_upsample              1000bc70 f   jdsample.obj
 0001:0000ad50       _fullsize_upsample         1000bd50 f   jdsample.obj
 0001:0000ad60       _noop_upsample             1000bd60 f   jdsample.obj
 0001:0000ad70       _int_upsample              1000bd70 f   jdsample.obj
 0001:0000ae70       _h2v1_upsample             1000be70 f   jdsample.obj
 0001:0000aed0       _h2v2_upsample             1000bed0 f   jdsample.obj
 0001:0000af50       _h2v1_fancy_upsample       1000bf50 f   jdsample.obj
 0001:0000b010       _h2v2_fancy_upsample       1000c010 f   jdsample.obj
 0001:0000b330       _error_exit                1000c330 f   jerror.obj
 0001:0000b350       _output_message            1000c350 f   jerror.obj
 0001:0000b350       _sun_jpeg_output_message   1000c350 f   jerror.obj
 0001:0000b390       _emit_message              1000c390 f   jerror.obj
 0001:0000b3d0       _format_message            1000c3d0 f   jerror.obj
 0001:0000b490       _reset_error_mgr           1000c490 f   jerror.obj
 0001:0000ca20       _alloc_small               1000da20 f   jmemmgr.obj
 0001:0000cb70       _alloc_large               1000db70 f   jmemmgr.obj
 0001:0000cc30       _alloc_sarray              1000dc30 f   jmemmgr.obj
 0001:0000cce0       _alloc_barray              1000dce0 f   jmemmgr.obj
 0001:0000cd90       _request_virt_sarray       1000dd90 f   jmemmgr.obj
 0001:0000ce00       _request_virt_barray       1000de00 f   jmemmgr.obj
 0001:0000ce70       _realize_virt_arrays       1000de70 f   jmemmgr.obj
 0001:0000d010       _do_sarray_io              1000e010 f   jmemmgr.obj
 0001:0000d0b0       _do_barray_io              1000e0b0 f   jmemmgr.obj
 0001:0000d150       _access_virt_sarray        1000e150 f   jmemmgr.obj
 0001:0000d2a0       _access_virt_barray        1000e2a0 f   jmemmgr.obj
 0001:0000d3f0       _free_pool                 1000e3f0 f   jmemmgr.obj
 0001:0000d4f0       _self_destruct             1000e4f0 f   jmemmgr.obj
 0001:0000d6b0       _start_pass_dcolor         1000e6b0 f   jmemnobs.obj
 0001:0000d6b0       _finish_pass_1_quant       1000e6b0 f   jmemnobs.obj
 0001:0000d6b0       _start_pass_downsample     1000e6b0 f   jmemnobs.obj
 0001:0000d6b0       _null_method               1000e6b0 f   jmemnobs.obj
 0001:0000d6b0       _finish_pass2              1000e6b0 f   jmemnobs.obj
 0001:0000d6c0       _select_ncolors            1000e6c0 f   jquant1.obj
 0001:0000d7b0       _create_colormap           1000e7b0 f   jquant1.obj
 0001:0000d930       _create_colorindex         1000e930 f   jquant1.obj
 0001:0000daa0       _make_odither_array        1000eaa0 f   jquant1.obj
 0001:0000db20       _create_odither_tables     1000eb20 f   jquant1.obj
 0001:0000db70       _color_quantize            1000eb70 f   jquant1.obj
 0001:0000dc20       _color_quantize3           1000ec20 f   jquant1.obj
 0001:0000dce0       _quantize_ord_dither       1000ece0 f   jquant1.obj
 0001:0000de10       _quantize3_ord_dither      1000ee10 f   jquant1.obj
 0001:0000df30       _quantize_fs_dither        1000ef30 f   jquant1.obj
 0001:0000e0f0       _alloc_fs_workspace        1000f0f0 f   jquant1.obj
 0001:0000e130       _start_pass_1_quant        1000f130 f   jquant1.obj
 0001:0000e220       _new_color_map_1_quant     1000f220 f   jquant1.obj
 0001:0000e2e0       _prescan_quantize          1000f2e0 f   jquant2.obj
 0001:0000e360       _update_box                1000f360 f   jquant2.obj
 0001:0000e750       _median_cut                1000f750 f   jquant2.obj
 0001:0000e8c0       _compute_color             1000f8c0 f   jquant2.obj
 0001:0000ea50       _select_colors             1000fa50 f   jquant2.obj
 0001:0000eae0       _find_nearby_colors        1000fae0 f   jquant2.obj
 0001:0000ecc0       _find_best_colors          1000fcc0 f   jquant2.obj
 0001:0000ee40       _fill_inverse_cmap         1000fe40 f   jquant2.obj
 0001:0000ef60       _pass2_no_dither           1000ff60 f   jquant2.obj
 0001:0000f030       _pass2_fs_dither           10010030 f   jquant2.obj
 0001:0000f320       _init_error_limit          10010320 f   jquant2.obj
 0001:0000f3c0       _finish_pass1              100103c0 f   jquant2.obj
 0001:0000f3f0       _start_pass_2_quant        100103f0 f   jquant2.obj
 0001:0000f520       _new_color_map_2_quant     10010520 f   jquant2.obj
 0001:0000fb40       _compress_data             10010b40 f   jccoefct.obj
 0001:0000fdf0       _compress_output           10010df0 f   jccoefct.obj
 0001:00010000       _compress_first_pass       10011000 f   jccoefct.obj
 0001:00010220       _start_pass_coef           10011220 f   jccoefct.obj
 0001:00010400       _rgb_ycc_start             10011400 f   jccolor.obj
 0001:000104e0       _rgb_ycc_convert           100114e0 f   jccolor.obj
 0001:00010600       _rgb_gray_convert          10011600 f   jccolor.obj
 0001:000106b0       _cmyk_ycck_convert         100116b0 f   jccolor.obj
 0001:00010810       _grayscale_convert         10011810 f   jccolor.obj
 0001:00010880       _null_convert              10011880 f   jccolor.obj
 0001:00010b40       _start_pass_fdctmgr        10011b40 f   jcdctmgr.obj
 0001:00010e40       _forward_DCT               10011e40 f   jcdctmgr.obj
 0001:00011210       _forward_DCT_float         10012210 f   jcdctmgr.obj
 0001:00011bb0       _emit_bits                 10012bb0 f   jchuff.obj
 0001:00011ca0       _encode_one_block          10012ca0 f   jchuff.obj
 0001:00011e30       _emit_restart              10012e30 f   jchuff.obj
 0001:00011f00       _encode_mcu_huff           10012f00 f   jchuff.obj
 0001:00012080       _finish_pass_huff          10013080 f   jchuff.obj
 0001:00012150       _htest_one_block           10013150 f   jchuff.obj
 0001:00012240       _encode_mcu_gather         10013240 f   jchuff.obj
 0001:00012570       _finish_pass_gather        10013570 f   jchuff.obj
 0001:00012680       _start_pass_huff           10013680 f   jchuff.obj
 0001:00012920       _process_data_simple_main  10013920 f   jcmainct.obj
 0001:000129d0       _start_pass_main           100139d0 f   jcmainct.obj
 0001:00012ab0       _emit_marker               10013ab0 f   jcmarker.obj
 0001:00012b20       _emit_2bytes               10013b20 f   jcmarker.obj
 0001:00012b90       _emit_dqt                  10013b90 f   jcmarker.obj
 0001:00012d20       _emit_dht                  10013d20 f   jcmarker.obj
 0001:00012e80       _emit_sof                  10013e80 f   jcmarker.obj
 0001:00013000       _emit_sos                  10014000 f   jcmarker.obj
 0001:000131e0       _emit_jfif_app0            100141e0 f   jcmarker.obj
 0001:00013400       _emit_adobe_app14          10014400 f   jcmarker.obj
 0001:00013570       _write_marker_header       10014570 f   jcmarker.obj
 0001:000135b0       _write_marker_byte         100145b0 f   jcmarker.obj
 0001:000135f0       _write_file_header         100145f0 f   jcmarker.obj
 0001:00013640       _write_frame_header        10014640 f   jcmarker.obj
 0001:00013730       _write_scan_header         10014730 f   jcmarker.obj
 0001:00013820       _write_file_trailer        10014820 f   jcmarker.obj
 0001:00013840       _write_tables_only         10014840 f   jcmarker.obj
 0001:000139a0       _initial_setup             100149a0 f   jcmaster.obj
 0001:00013b70       _validate_script           10014b70 f   jcmaster.obj
 0001:00013f30       _select_scan_parameters    10014f30 f   jcmaster.obj
 0001:00014020       _per_scan_setup            10015020 f   jcmaster.obj
 0001:000141f0       _prepare_for_pass          100151f0 f   jcmaster.obj
 0001:00014390       _pass_startup              10015390 f   jcmaster.obj
 0001:000143c0       _finish_pass_master        100153c0 f   jcmaster.obj
 0001:000146e0       _add_huff_table            100156e0 f   jcparam.obj
 0001:00014790       _std_huff_tables           10015790 f   jcparam.obj
 0001:00014ad0       _fill_dc_scans             10015ad0 f   jcparam.obj
 0001:00015170       _emit_bits                 10016170 f   jcphuff.obj
 0001:000152b0       _emit_buffered_bits        100162b0 f   jcphuff.obj
 0001:000152e0       _emit_eobrun               100162e0 f   jcphuff.obj
 0001:00015380       _emit_restart              10016380 f   jcphuff.obj
 0001:00015490       _encode_mcu_DC_first       10016490 f   jcphuff.obj
 0001:00015610       _encode_mcu_AC_first       10016610 f   jcphuff.obj
 0001:00015810       _encode_mcu_DC_refine      10016810 f   jcphuff.obj
 0001:000158e0       _encode_mcu_AC_refine      100168e0 f   jcphuff.obj
 0001:00015b80       _finish_pass_phuff         10016b80 f   jcphuff.obj
 0001:00015bd0       _finish_pass_gather_phuff  10016bd0 f   jcphuff.obj
 0001:00015cc0       _start_pass_phuff          10016cc0 f   jcphuff.obj
 0001:00015e90       _start_pass_prep           10016e90 f   jcprepct.obj
 0001:00015ee0       _pre_process_data          10016ee0 f   jcprepct.obj
 0001:000160f0       _pre_process_context       100170f0 f   jcprepct.obj
 0001:00016310       _create_context_buffer     10017310 f   jcprepct.obj
 0001:00016510       _expand_right_edge         10017510 f   jcsample.obj
 0001:00016570       _sep_downsample            10017570 f   jcsample.obj
 0001:00016600       _int_downsample            10017600 f   jcsample.obj
 0001:00016730       _fullsize_downsample       10017730 f   jcsample.obj
 0001:00016780       _h2v1_downsample           10017780 f   jcsample.obj
 0001:00016820       _h2v2_downsample           10017820 f   jcsample.obj
 0001:00016900       _h2v2_smooth_downsample    10017900 f   jcsample.obj
 0001:00016b90       _fullsize_smooth_downsample 10017b90 f   jcsample.obj
